:10000000830100308A0004282030840025300F202E
:1000100083010A128A11F92F04068001840A04065A
:06002000031D0C28003452
:100F8400FF308301A10703110318013E031DA207CB
:100F9400FF3003110318013E031DA307FF300311A3
:100FA4000318013E031DA40724082304220421047A
:100FB40003190800C22F8301A100831203130C1E1E
:100FC400DF2F21089900080083018C1EE62F1A08E0
:100FD40008008316031307138717903083129800B1
:100FE4002430831698008130990083120800EB277F
:0C0FF400E627A000DD272A30DD27FA2FB9
:02400E00323F3F
:00000001FF
